:100000000EC026C025C05AC023C022C021C020C0B7
:100010001FC01EC01DC01CC01BC01AC019C01124A7
:100020001FBECFEDCDBF10E0A0E6B0E0E4EDF6E0FE
:1000300002C005900D92A836B107D9F720E0A8E6D6
:10004000B0E001C01D92AC39B207E1F734D140C332
:10005000D7CF81E087B9369A3699FECF24B135B132
:1000600080919B00803110F010929B008091710074
:1000700090917200A0917300B091740060919B0008
:10008000E62FF0E0EE0FFF1FEB58FF4F408151814C
:1000900031832083820F931FA11DB11D841B950BFB
:1000A000A109B1098093710090937200A09373002D
:1000B000B09374006F5F60939B0008951F920F923E
:1000C0000FB60F9211242F934F935F936F937F93EB
:1000D0008F939F93AF93BF9380916800882309F417
:1000E00055C08091690090916A00A0916B00B09119
:1000F0006C008F3F9105A105B10509F010F4AC012A
:100100000FC08F3F21E09207A105B10538F4AC0183
:10011000BD01769567955795479502C04FEF50E022
:10012000841B950BA109B1098093690090936A0023
:10013000A0936B00B0936C002EB5240F2EBD892BBD
:100140008A2B8B2B09F0A9C080B78F7E80BF80914E
:10015000600090916100A0916200B09163004091B5
:100160006400509165006091660070916700841B87
:10017000950BA60BB70B80936D0090936E00A09328
:100180006F00B09370001092680087C080916D007E
:1001900090916E00A0916F00B09170008F3F91051B
:1001A000A105B10509F010F4AC010FC08F3F21E0AB
:1001B0009207A105B10538F4AC01BD0176956795AC
:1001C0005795479502C04FEF50E0841B950BA1094E
:1001D000B10980936D0090936E00A0936F00B0936F
:1001E00070002EB5240F2EBD892B8A2B8B2B09F086
:1001F00054C081E080936800809164009091650014
:10020000A0916600B09167008093690090936A00A6
:10021000A0936B00B0936C0080919500882319F037
:1002200080B7806180BF80919600882331F18091F2
:10023000970090919800A0919900B0919A008093B6
:10024000600090936100A0936200B093630080917E
:10025000970090919800A0919900B0919A00B6955E
:10026000A795979587958093640090936500A093D8
:100270006600B093670010929600809160009091A4
:100280006100A0916200B091630080936D00909333
:100290006E00A0936F00B0937000BF91AF919F91DB
:1002A0008F917F916F915F914F912F910F900FBE22
:1002B0000F901F90189580E886BD16BCB99A89E109
:1002C00088BB81E280BF80E488BF89B7806489BF32
:1002D00087E886B97894C1E0BCDE809196008111F0
:1002E000FBCF6091710070917200809173009091CA
:1002F0007400D1D020E030E040E85DE37ED120E022
:1003000030EC4FE754E433D09F7720E030E44CE901
:1003100055E473D1F62E072F182FD92F20E030E0A7
:1003200040EA50E420D087FF07C010929500F12CDE
:1003300000E010EAD0E402C0C09395002F2D302FCA
:10034000412F5D2F60E074E284EF9AE410D077D003
:1003500060939700709398008093990090939A000F
:10036000C0939600B9CFD4D008F481E008950CD0A2
:100370000AC102D140F0F9D030F021F45F3F19F00A
:10038000EBC0511134C1EEC00FD198F39923C9F3DA
:100390005523B1F3951B550BBB27AA27621773078B
:1003A000840738F09F5F5F4F220F331F441FAA1F3F
:1003B000A9F333D00E2E3AF0E0E830D091505040FF
:1003C000E695001CCAF729D0FE2F27D0660F771FAD
:1003D000881FBB1F261737074807AB07B0E809F08F
:1003E000BB0B802DBF01FF2793585F4F2AF09E3F24
:1003F000510568F0B1C0FBC05F3FECF3983EDCF301
:10040000869577956795B795F7959F5FC9F7880F9C
:10041000911D9695879597F90895E1E0660F771FEE
:10042000881FBB1F621773078407BA0720F0621B7F
:10043000730B840BBA0BEE1F88F7E0950895BCD0C0
:1004400088F09F5790F0B92F9927B751A0F0D1F0BD
:10045000660F771F881F991F1AF0BA95C9F712C047
:10046000B13081F0C3D0B1E00895C0C0672F782FBC
:100470008827B85F39F0B93FCCF3869577956795B3
:10048000B395D9F73EF490958095709561957F4F1F
:100490008F4F9F4F0895E89409C097FB3EF49095C5
:1004A0008095709561957F4F8F4F9F4F9923A9F04D
:1004B000F92F96E9BB279395F695879577956795DC
:1004C000B795F111F8CFFAF4BB0F11F460FF1BC020
:1004D0006F5F7F4F8F4F9F4F16C0882311F096E9B3
:1004E00011C0772321F09EE8872F762F05C0662361
:1004F00071F096E8862F70E060E02AF09A95660F1A
:10050000771F881FDAF7880F9695879597F90895D2
:10051000990F0008550FAA0BE0E8FEEF1616170614
:10052000E807F907C0F012161306E407F50798F07C
:10053000621B730B840B950B39F40A2661F0232B95
:10054000242B252B21F408950A2609F4A140A69511
:100550008FEF811D811D089597F99F6780E870E0F6
:1005600060E008959FEF80EC089500240A94161629
:10057000170618060906089500240A941216130691
:10058000140605060895092E0394000C11F488231F
:1005900052F0BB0F40F4BF2B11F460FF04C06F5F3B
:1005A0007F4F8F4F9F4F089557FD9058440F551F11
:1005B00059F05F3F71F04795880F97FB991F61F0E5
:1005C0009F3F79F087950895121613061406551F5C
:1005D000F2CF4695F1DF08C0161617061806991FC8
:1005E000F1CF86957105610508940895E894BB27BD
:1005F00066277727CB0197F908950AD0C4CFB5DFD6
:1006000028F0BADF18F0952309F0A6CFABCFEFCFD3
:10061000CBDFA8F39923D9F35523C9F3950F50E005
:10062000551FAA27EE27FF27BB27002408946795AC
:1006300020F4E20FF31FB41F0A1E220F331F441FC2
:10064000AA1F6695A9F7779530F4F30FB41F0A1E19
:10065000121E08F46395330F441FAA1F221F7695BC
:1006600099F7879520F4B40F0A1E121E631F440FDA
:10067000AA1F221F331F8695A9F7862F712D602D83
:1006800011249F5750408AF0E1F088234AF0EE0F82
:10069000FF1FBB1F661F771F881F91505040A9F78F
:1006A0009E3F510570F058CFA2CF5F3FECF3983ECC
:1006B000DCF3869577956795B795F795E7959F5FF6
:1006C000C1F7FE2B880F911D9695879597F9089590
:0406D000F894FFCFCC
:0806D400D0070000E80300005C
:00000001FF
